 csp_serial

 Timestamp is 4fb04cb5 (Mon May 14 12:07:17 2012)

 Preferred load address is 10000000

 Start         Length     Name                   Class
 0001:00000000 00000004H .CRT$XCA                CODE
 0001:00000004 00000004H .CRT$XCZ                CODE
 0001:00000008 00000004H .CRT$XIA                CODE
 0001:0000000c 00000004H .CRT$XIZ                CODE
 0001:00000010 00000004H .CRT$XPA                CODE
 0001:00000014 00000004H .CRT$XPZ                CODE
 0001:00000018 00000004H .CRT$XTA                CODE
 0001:0000001c 00000004H .CRT$XTZ                CODE
 0001:00000020 000002baH .rdata                  CODE
 0001:000002dc 00000027H .rdata$debug            CODE
 0001:00000304 0000610cH .text                   CODE
 0001:00006410 00000220H .xdata                  CODE
 0001:00006630 0000003cH .idata$2                CODE
 0001:0000666c 00000014H .idata$3                CODE
 0001:00006680 00000110H .idata$4                CODE
 0001:00006790 00000166H .idata$6                CODE
 0001:00006900 00000136H .edata                  CODE
 0002:00000000 00000110H .idata$5                DATA
 0002:00000110 00000008H .data                   DATA
 0002:00000118 0000001cH .bss                    DATA
 0003:00000000 000003e8H .pdata                  DATA

  Address         Publics by Value              Rva+Base       Lib:Object

 0000:00000000       ___safe_se_handler_count   00000000     <absolute>
 0000:00000000       ___safe_se_handler_table   00000000     <absolute>
 0001:00000000       __xc_a                     10001000     corelib0:crt0init.obj
 0001:00000004       __xc_z                     10001004     corelib0:crt0init.obj
 0001:00000008       __xi_a                     10001008     corelib0:crt0init.obj
 0001:0000000c       __xi_z                     1000100c     corelib0:crt0init.obj
 0001:00000010       __xp_a                     10001010     corelib0:crt0init.obj
 0001:00000014       __xp_z                     10001014     corelib0:crt0init.obj
 0001:00000018       __xt_a                     10001018     corelib0:crt0init.obj
 0001:0000001c       __xt_z                     1000101c     corelib0:crt0init.obj
 0001:000000d0       ??_C@_1BI@BHLBGEOK@?$AAP?$AAr?$AAi?$AAo?$AAr?$AAi?$AAt?$AAy?$AA2?$AA5?$AA6?$AA?$AA@ 100010d0     com_mdd2:mdd.obj
 0001:000000e8       ??_C@_1CC@KMPFMANC@?$AAD?$AAe?$AAv?$AAi?$AAc?$AAe?$AAA?$AAr?$AAr?$AAa?$AAy?$AAI?$AAn?$AAd?$AAe?$AAx?$AA?$AA@ 100010e8     com_mdd2:mdd.obj
 0001:000001d0       IoVTbl                     100011d0     serial_common_topaz_v1:serial.obj
 0001:00000248       IrVTbl                     10001248     serial_common_topaz_v1:serial.obj
 0001:000002c0       ??_C@_1M@PEPOCCHH@?$AAI?$AAo?$AAL?$AAe?$AAn?$AA?$AA@ 100012c0     serial_common_topaz_v1:serial.obj
 0001:000002cc       ??_C@_1O@JMCNHCBG@?$AAI?$AAo?$AAB?$AAa?$AAs?$AAe?$AA?$AA@ 100012cc     serial_common_topaz_v1:serial.obj
 0001:00000304       BSPUartCalRFDIV            10001304 f   bspserial.obj
 0001:0000038c       BSPUartGetType             1000138c f   bspserial.obj
 0001:000003ec       BSPUartEnableClock         100013ec f   bspserial.obj
 0001:00000484       BSPUartConfigTranceiver    10001484 f   bspserial.obj
 0001:00000488       BSPUartConfigureGPIO       10001488 f   bspserial.obj
 0001:00000924       BSPSerGetChannelPriority   10001924 f   bspserial.obj
 0001:0000092c       BSPSerGetDMAIsEnabled      1000192c f   bspserial.obj
 0001:0000098c       BSPSerGetDMARequest        1000198c f   bspserial.obj
 0001:00000a38       BSPSerAcquireDMAReqGpr     10001a38 f   bspserial.obj
 0001:00000a40       BSPSerRestoreDMAReqGpr     10001a40 f   bspserial.obj
 0001:00000a48       GetSdmaChannelIRQ          10001a48 f   bspserial.obj
 0001:00000a50       BSPGetDMABuffSize          10001a50 f   bspserial.obj
 0001:00000a64       DllEntry                   10001a64 f   com_mdd2:mdd.obj
 0001:00000a7c       DoTxData                   10001a7c f   com_mdd2:mdd.obj
 0001:00000ba0       StopDispatchThread         10001ba0 f   com_mdd2:mdd.obj
 0001:00000c34       ApplyDCB                   10001c34 f   com_mdd2:mdd.obj
 0001:00000ee0       COM_PreClose               10001ee0 f   com_mdd2:mdd.obj
 0001:00000fa4       COM_Close                  10001fa4 f   com_mdd2:mdd.obj
 0001:000010c8       ProcessExiting             100020c8 f   com_mdd2:mdd.obj
 0001:000010fc       COM_PreDeinit              100020fc f   com_mdd2:mdd.obj
 0001:0000118c       COM_Deinit                 1000218c f   com_mdd2:mdd.obj
 0001:000012b4       COM_Read                   100022b4 f   com_mdd2:mdd.obj
 0001:00001610       COM_Seek                   10002610 f   com_mdd2:mdd.obj
 0001:00001618       COM_PowerUp                10002618 f   com_mdd2:mdd.obj
 0001:00001658       COM_PowerDown              10002658 f   com_mdd2:mdd.obj
 0001:000016a0       WaitCommEvent_mdd          100026a0 f   com_mdd2:mdd.obj
 0001:000017f4       EvaluateEventFlag          100027f4 f   com_mdd2:mdd.obj
 0001:0000189c       COM_IOControl              1000289c f   com_mdd2:mdd.obj
 0001:00002244       SerialEventHandler         10003244 f   com_mdd2:mdd.obj
 0001:00002618       StartDispatchThread        10003618 f   com_mdd2:mdd.obj
 0001:000026a8       COM_Init                   100036a8 f   com_mdd2:mdd.obj
 0001:00002944       COM_Open                   10003944 f   com_mdd2:mdd.obj
 0001:00002bf0       COM_Write                  10003bf0 f   com_mdd2:mdd.obj
 0001:00002da8       EventModify                10003da8 f   coredll:COREDLL.dll
 0001:00002db8       DisableThreadLibraryCalls  10003db8 f   coredll:COREDLL.dll
 0001:00002dc8       LeaveCriticalSection       10003dc8 f   coredll:COREDLL.dll
 0001:00002dd8       EnterCriticalSection       10003dd8 f   coredll:COREDLL.dll
 0001:00002de8       InterruptDisable           10003de8 f   coredll:COREDLL.dll
 0001:00002df8       InterruptDone              10003df8 f   coredll:COREDLL.dll
 0001:00002e08       CloseHandle                10003e08 f   coredll:COREDLL.dll
 0001:00002e18       Sleep                      10003e18 f   coredll:COREDLL.dll
 0001:00002e28       WaitForSingleObject        10003e28 f   coredll:COREDLL.dll
 0001:00002e38       CeSetThreadPriority        10003e38 f   coredll:COREDLL.dll
 0001:00002e48       CeGetThreadPriority        10003e48 f   coredll:COREDLL.dll
 0001:00002e58       SetLastError               10003e58 f   coredll:COREDLL.dll
 0001:00002e68       LocalFree                  10003e68 f   coredll:COREDLL.dll
 0001:00002e78       DeleteCriticalSection      10003e78 f   coredll:COREDLL.dll
 0001:00002e88       SetThreadPriority          10003e88 f   coredll:COREDLL.dll
 0001:00002e98       InterlockedDecrement       10003e98 f   coredll:COREDLL.dll
 0001:00002ea8       GetTickCount               10003ea8 f   coredll:COREDLL.dll
 0001:00002eb8       CeSafeCopyMemory           10003eb8 f   coredll:COREDLL.dll
 0001:00002ec8       InterlockedIncrement       10003ec8 f   coredll:COREDLL.dll
 0001:00002ed8       InterlockedExchange        10003ed8 f   coredll:COREDLL.dll
 0001:00002ee8       InterlockedCompareExchange 10003ee8 f   coredll:COREDLL.dll
 0001:00002ef8       ExitThread                 10003ef8 f   coredll:COREDLL.dll
 0001:00002f08       CreateThread               10003f08 f   coredll:COREDLL.dll
 0001:00002f18       InterruptInitialize        10003f18 f   coredll:COREDLL.dll
 0001:00002f28       RegCloseKey                10003f28 f   coredll:COREDLL.dll
 0001:00002f38       RegQueryValueExW           10003f38 f   coredll:COREDLL.dll
 0001:00002f48       OpenDeviceKey              10003f48 f   coredll:COREDLL.dll
 0001:00002f58       CreateEventW               10003f58 f   coredll:COREDLL.dll
 0001:00002f68       InitializeCriticalSection  10003f68 f   coredll:COREDLL.dll
 0001:00002f78       LocalAlloc                 10003f78 f   coredll:COREDLL.dll
 0001:00002f88       CeFreeAsynchronousBuffer   10003f88 f   coredll:COREDLL.dll
 0001:00002f98       CeAllocAsynchronousBuffer  10003f98 f   coredll:COREDLL.dll
 0001:00002fa8       DDKClockGetFreq            10003fa8 f   cspddk:CSPDDK.dll
 0001:00002fb8       DDKClockSetGatingMode      10003fb8 f   cspddk:CSPDDK.dll
 0001:00002fc8       DDKIomuxSelectInput        10003fc8 f   cspddk:CSPDDK.dll
 0001:00002fd8       DDKIomuxSetPadConfig       10003fd8 f   cspddk:CSPDDK.dll
 0001:00002fe8       DDKIomuxSetPinMux          10003fe8 f   cspddk:CSPDDK.dll
 0001:00002ff8       _DllEntryCRTStartup        10003ff8 f   corelib0:pegdentry.obj
 0001:00003040       __GSHandlerCheckCommon     10004040 f   corelib0:gshandler.obj
 0001:0000307c       __GSHandlerCheck           1000407c f   corelib0:gshandler.obj
 0001:000030a0       __security_init_cookie     100040a0 f   corelib0:seccinit.obj
 0001:000030fc       __security_check_cookie    100040fc f   corelib0:armsecgs.obj
 0001:00003110       __gsfailure                10004110 f   corelib0:armsecgs.obj
 0001:00003250       _cexit                     10004250 f   corelib0:cexit.obj
 0001:0000326c       _initterm                  1000426c f   corelib0:crt0dat.obj
 0001:000032a0       _cinit                     100042a0 f   corelib0:crt0dat.obj
 0001:000032d4       __rt_udiv                  100042d4 f   corelib1:COREDLL.dll
 0001:000032e4       memcpy                     100042e4 f   corelib1:COREDLL.dll
 0001:000032f4       __C_specific_handler       100042f4 f   corelib1:COREDLL.dll
 0001:00003304       memset                     10004304 f   corelib1:COREDLL.dll
 0001:00003314       memmove                    10004314 f   corelib1:COREDLL.dll
 0001:00003324       __security_gen_cookie2     10004324 f   corelib1:COREDLL.dll
 0001:00003334       __report_gsfailure         10004334 f   corelib1:COREDLL.dll
 0001:00003344       free                       10004344 f   corelib1:COREDLL.dll
 0001:00003354       MapDMABuffers              10004354 f   serial_common_topaz_v1:serial.obj
 0001:000033f8       UnmapDMABuffers            100043f8 f   serial_common_topaz_v1:serial.obj
 0001:00003488       DeinitChannelDMA           10004488 f   serial_common_topaz_v1:serial.obj
 0001:000034c8       InitChannelDMA             100044c8 f   serial_common_topaz_v1:serial.obj
 0001:00003544       InitDMA                    10004544 f   serial_common_topaz_v1:serial.obj
 0001:000035c8       DeInitDMA                  100045c8 f   serial_common_topaz_v1:serial.obj
 0001:00003c58       GetSerialObject            10004c58 f   serial_common_topaz_v1:serial.obj
 0001:00003cb0       SL_ReadModemStatus         10004cb0 f   serial_common_topaz_v1:serialhw.obj
 0001:00003ddc       SL_ReadLineStatus          10004ddc f   serial_common_topaz_v1:serialhw.obj
 0001:00003f1c       SL_SetOutputMode           10004f1c f   serial_common_topaz_v1:serialhw.obj
 0001:00003f98       SL_ClearPendingInts        10004f98 f   serial_common_topaz_v1:serialhw.obj
 0001:00004018       SL_SetStopBits             10005018 f   serial_common_topaz_v1:serialhw.obj
 0001:0000412c       SL_SetBaudRate             1000512c f   serial_common_topaz_v1:serialhw.obj
 0001:00004254       SL_SetByteSize             10005254 f   serial_common_topaz_v1:serialhw.obj
 0001:00004360       SL_SetParity               10005360 f   serial_common_topaz_v1:serialhw.obj
 0001:000044ac       SL_SetFlowControl          100054ac f   serial_common_topaz_v1:serialhw.obj
 0001:00004594       SL_Reset                   10005594 f   serial_common_topaz_v1:serialhw.obj
 0001:000046ac       SL_Init                    100056ac f   serial_common_topaz_v1:serialhw.obj
 0001:00004720       SL_Deinit                  10005720 f   serial_common_topaz_v1:serialhw.obj
 0001:000047f4       SL_Open                    100057f4 f   serial_common_topaz_v1:serialhw.obj
 0001:00004ba8       SL_Close                   10005ba8 f   serial_common_topaz_v1:serialhw.obj
 0001:00004dac       SL_PowerOff                10005dac f   serial_common_topaz_v1:serialhw.obj
 0001:00004dc4       SL_PowerOn                 10005dc4 f   serial_common_topaz_v1:serialhw.obj
 0001:00004dec       SL_GetIntrType             10005dec f   serial_common_topaz_v1:serialhw.obj
 0001:000050a8       SL_RxIntrHandler           100060a8 f   serial_common_topaz_v1:serialhw.obj
 0001:00005498       SL_TxIntrHandler           10006498 f   serial_common_topaz_v1:serialhw.obj
 0001:00005880       SL_ModemIntrHandler        10006880 f   serial_common_topaz_v1:serialhw.obj
 0001:000059d0       SL_LineIntrHandler         100069d0 f   serial_common_topaz_v1:serialhw.obj
 0001:000059e0       SL_GetRxBufferSize         100069e0 f   serial_common_topaz_v1:serialhw.obj
 0001:000059f0       SL_ClearDTR                100069f0 f   serial_common_topaz_v1:serialhw.obj
 0001:00005a64       SL_SetDTR                  10006a64 f   serial_common_topaz_v1:serialhw.obj
 0001:00005ad8       SL_ClearRTS                10006ad8 f   serial_common_topaz_v1:serialhw.obj
 0001:00005b74       SL_SetRTS                  10006b74 f   serial_common_topaz_v1:serialhw.obj
 0001:00005c28       SL_ClearBreak              10006c28 f   serial_common_topaz_v1:serialhw.obj
 0001:00005c9c       SL_SetBreak                10006c9c f   serial_common_topaz_v1:serialhw.obj
 0001:00005d10       SL_XmitComChar             10006d10 f   serial_common_topaz_v1:serialhw.obj
 0001:00005df0       SL_GetStatus               10006df0 f   serial_common_topaz_v1:serialhw.obj
 0001:00005ea8       SL_GetModemStatus          10006ea8 f   serial_common_topaz_v1:serialhw.obj
 0001:00005f08       SL_PurgeComm               10006f08 f   serial_common_topaz_v1:serialhw.obj
 0001:00005f60       SL_SetDCB                  10006f60 f   serial_common_topaz_v1:serialhw.obj
 0001:000060b8       SL_SetCommTimeouts         100070b8 f   serial_common_topaz_v1:serialhw.obj
 0001:000060d4       SL_Ioctl                   100070d4 f   serial_common_topaz_v1:serialhw.obj
 0001:000062d0       HalAllocateCommonBuffer    100072d0 f   ceddk:CEDDK.dll
 0001:000062e0       HalFreeCommonBuffer        100072e0 f   ceddk:CEDDK.dll
 0001:000062f0       MmMapIoSpace               100072f0 f   ceddk:CEDDK.dll
 0001:00006300       HalTranslateBusAddress     10007300 f   ceddk:CEDDK.dll
 0001:00006310       MmUnmapIoSpace             10007310 f   ceddk:CEDDK.dll
 0001:00006320       TerminateProcess           10007320 f   coredll:COREDLL.dll
 0001:00006330       KernelIoControl            10007330 f   coredll:COREDLL.dll
 0001:00006340       CeEventHasOccurred         10007340 f   coredll:COREDLL.dll
 0001:00006350       IsAPIReady                 10007350 f   coredll:COREDLL.dll
 0001:00006360       DDKSdmaCloseChan           10007360 f   cspddk:CSPDDK.dll
 0001:00006370       DDKSdmaAllocChain          10007370 f   cspddk:CSPDDK.dll
 0001:00006380       DDKSdmaOpenChan            10007380 f   cspddk:CSPDDK.dll
 0001:00006390       DDKSdmaStartChan           10007390 f   cspddk:CSPDDK.dll
 0001:000063a0       DDKSdmaSetBufDesc          100073a0 f   cspddk:CSPDDK.dll
 0001:000063b0       DDKSdmaClearChainStatus    100073b0 f   cspddk:CSPDDK.dll
 0001:000063c0       DDKSdmaInitChain           100073c0 f   cspddk:CSPDDK.dll
 0001:000063d0       DDKSdmaStopChan            100073d0 f   cspddk:CSPDDK.dll
 0001:000063e0       DDKSdmaGetBufDescStatus    100073e0 f   cspddk:CSPDDK.dll
 0001:000063f0       DDKSdmaClearBufDescStatus  100073f0 f   cspddk:CSPDDK.dll
 0001:00006400       __rt_udiv64by64            10007400 f   corelib1:COREDLL.dll
 0001:00006630       __IMPORT_DESCRIPTOR_COREDLL 10007630     coredll:COREDLL.dll
 0001:00006644       __IMPORT_DESCRIPTOR_CSPDDK 10007644     cspddk:CSPDDK.dll
 0001:00006658       __IMPORT_DESCRIPTOR_CEDDK  10007658     ceddk:CEDDK.dll
 0001:0000666c       __NULL_IMPORT_DESCRIPTOR   1000766c     coredll:COREDLL.dll
 0002:00000000       __imp_MmUnmapIoSpace       10008000     ceddk:CEDDK.dll
 0002:00000004       __imp_MmMapIoSpace         10008004     ceddk:CEDDK.dll
 0002:00000008       __imp_HalFreeCommonBuffer  10008008     ceddk:CEDDK.dll
 0002:0000000c       __imp_HalAllocateCommonBuffer 1000800c     ceddk:CEDDK.dll
 0002:00000010       __imp_HalTranslateBusAddress 10008010     ceddk:CEDDK.dll
 0002:00000014       \177CEDDK_NULL_THUNK_DATA  10008014     ceddk:CEDDK.dll
 0002:00000018       __imp_CloseHandle          10008018     coredll:COREDLL.dll
 0002:0000001c       __imp_Sleep                1000801c     coredll:COREDLL.dll
 0002:00000020       __imp_WaitForSingleObject  10008020     coredll:COREDLL.dll
 0002:00000024       __imp_CeSetThreadPriority  10008024     coredll:COREDLL.dll
 0002:00000028       __imp_CeGetThreadPriority  10008028     coredll:COREDLL.dll
 0002:0000002c       __imp_SetLastError         1000802c     coredll:COREDLL.dll
 0002:00000030       __imp_LocalFree            10008030     coredll:COREDLL.dll
 0002:00000034       __imp_DeleteCriticalSection 10008034     coredll:COREDLL.dll
 0002:00000038       __imp_SetThreadPriority    10008038     coredll:COREDLL.dll
 0002:0000003c       __imp_InterlockedDecrement 1000803c     coredll:COREDLL.dll
 0002:00000040       __imp_GetTickCount         10008040     coredll:COREDLL.dll
 0002:00000044       __imp_CeSafeCopyMemory     10008044     coredll:COREDLL.dll
 0002:00000048       __imp_InterlockedIncrement 10008048     coredll:COREDLL.dll
 0002:0000004c       __imp_InterlockedExchange  1000804c     coredll:COREDLL.dll
 0002:00000050       __imp_InterlockedCompareExchange 10008050     coredll:COREDLL.dll
 0002:00000054       __imp_ExitThread           10008054     coredll:COREDLL.dll
 0002:00000058       __imp_CreateThread         10008058     coredll:COREDLL.dll
 0002:0000005c       __imp_InterruptInitialize  1000805c     coredll:COREDLL.dll
 0002:00000060       __imp_RegCloseKey          10008060     coredll:COREDLL.dll
 0002:00000064       __imp_RegQueryValueExW     10008064     coredll:COREDLL.dll
 0002:00000068       __imp_OpenDeviceKey        10008068     coredll:COREDLL.dll
 0002:0000006c       __imp_InterruptDone        1000806c     coredll:COREDLL.dll
 0002:00000070       __imp_InitializeCriticalSection 10008070     coredll:COREDLL.dll
 0002:00000074       __imp_LocalAlloc           10008074     coredll:COREDLL.dll
 0002:00000078       __imp_CeFreeAsynchronousBuffer 10008078     coredll:COREDLL.dll
 0002:0000007c       __imp_CeAllocAsynchronousBuffer 1000807c     coredll:COREDLL.dll
 0002:00000080       __imp_IsAPIReady           10008080     coredll:COREDLL.dll
 0002:00000084       __imp_CeEventHasOccurred   10008084     coredll:COREDLL.dll
 0002:00000088       __imp___rt_udiv64by64      10008088     corelib1:COREDLL.dll
 0002:0000008c       __imp_KernelIoControl      1000808c     coredll:COREDLL.dll
 0002:00000090       __imp_TerminateProcess     10008090     coredll:COREDLL.dll
 0002:00000094       __imp_InterruptDisable     10008094     coredll:COREDLL.dll
 0002:00000098       __imp___rt_udiv            10008098     corelib1:COREDLL.dll
 0002:0000009c       __imp_memcpy               1000809c     corelib1:COREDLL.dll
 0002:000000a0       __imp___C_specific_handler 100080a0     corelib1:COREDLL.dll
 0002:000000a4       __imp_memset               100080a4     corelib1:COREDLL.dll
 0002:000000a8       __imp_memmove              100080a8     corelib1:COREDLL.dll
 0002:000000ac       __imp___security_gen_cookie2 100080ac     corelib1:COREDLL.dll
 0002:000000b0       __imp___report_gsfailure   100080b0     corelib1:COREDLL.dll
 0002:000000b4       __imp_free                 100080b4     corelib1:COREDLL.dll
 0002:000000b8       __imp_EnterCriticalSection 100080b8     coredll:COREDLL.dll
 0002:000000bc       __imp_LeaveCriticalSection 100080bc     coredll:COREDLL.dll
 0002:000000c0       __imp_DisableThreadLibraryCalls 100080c0     coredll:COREDLL.dll
 0002:000000c4       __imp_CreateEventW         100080c4     coredll:COREDLL.dll
 0002:000000c8       __imp_EventModify          100080c8     coredll:COREDLL.dll
 0002:000000cc       \177COREDLL_NULL_THUNK_DATA 100080cc     coredll:COREDLL.dll
 0002:000000d0       __imp_DDKIomuxSetPinMux    100080d0     cspddk:CSPDDK.dll
 0002:000000d4       __imp_DDKIomuxSetPadConfig 100080d4     cspddk:CSPDDK.dll
 0002:000000d8       __imp_DDKClockSetGatingMode 100080d8     cspddk:CSPDDK.dll
 0002:000000dc       __imp_DDKClockGetFreq      100080dc     cspddk:CSPDDK.dll
 0002:000000e0       __imp_DDKSdmaCloseChan     100080e0     cspddk:CSPDDK.dll
 0002:000000e4       __imp_DDKSdmaAllocChain    100080e4     cspddk:CSPDDK.dll
 0002:000000e8       __imp_DDKSdmaOpenChan      100080e8     cspddk:CSPDDK.dll
 0002:000000ec       __imp_DDKSdmaStartChan     100080ec     cspddk:CSPDDK.dll
 0002:000000f0       __imp_DDKSdmaSetBufDesc    100080f0     cspddk:CSPDDK.dll
 0002:000000f4       __imp_DDKSdmaClearChainStatus 100080f4     cspddk:CSPDDK.dll
 0002:000000f8       __imp_DDKSdmaInitChain     100080f8     cspddk:CSPDDK.dll
 0002:000000fc       __imp_DDKSdmaStopChan      100080fc     cspddk:CSPDDK.dll
 0002:00000100       __imp_DDKSdmaGetBufDescStatus 10008100     cspddk:CSPDDK.dll
 0002:00000104       __imp_DDKSdmaClearBufDescStatus 10008104     cspddk:CSPDDK.dll
 0002:00000108       __imp_DDKIomuxSelectInput  10008108     cspddk:CSPDDK.dll
 0002:0000010c       \177CSPDDK_NULL_THUNK_DATA 1000810c     cspddk:CSPDDK.dll
 0002:00000110       __security_cookie          10008110     corelib0:seccinit.obj
 0002:00000114       __security_cookie_complement 10008114     corelib0:seccinit.obj
 0002:0000011c       _exitflag                  1000811c     corelib0:cexit.obj
 0002:00000128       __onexitend                10008128     <common>
 0002:0000012c       __onexitbegin              1000812c     <common>
 0002:00000130       g_pcsExit                  10008130     <common>

 entry point at        0001:00002ff8

 Static symbols

 0001:000025ac       SerialDispatchThread       100035ac f   com_mdd2:mdd.obj
 0001:00003154       doexit                     10004154 f   corelib0:cexit.obj
 0001:00003610       Ser_GetRegistryData        10004610 f   serial_common_topaz_v1:serial.obj
 0001:000036f8       SerInit                    100046f8 f   serial_common_topaz_v1:serial.obj
 0001:000039d0       SerSerialInit              100049d0 f   serial_common_topaz_v1:serial.obj
 0001:000039f0       SerIRInit                  100049f0 f   serial_common_topaz_v1:serial.obj
 0001:00003a10       SerPostInit                10004a10 f   serial_common_topaz_v1:serial.obj
 0001:00003a24       SerOpen                    10004a24 f   serial_common_topaz_v1:serial.obj
 0001:00003a80       SerClose                   10004a80 f   serial_common_topaz_v1:serial.obj
 0001:00003ae4       SerDeinit                  10004ae4 f   serial_common_topaz_v1:serial.obj
 0001:00003b94       SerPowerOff                10004b94 f   serial_common_topaz_v1:serial.obj
 0001:00003bbc       SerPowerOn                 10004bbc f   serial_common_topaz_v1:serial.obj
 0001:00003bf0       SerEnableIR                10004bf0 f   serial_common_topaz_v1:serial.obj
 0001:00003c14       SerDisableIR               10004c14 f   serial_common_topaz_v1:serial.obj
 0001:00003c38       SerGetCommProperties       10004c38 f   serial_common_topaz_v1:serial.obj
